:0200000480007A
:100000006F008004732F2034930F80006308FF0378
:10001000930F90006304FF03930FB0006300FF038E
:10002000130F000063040F0067000F00732F2034CC
:1000300063540F006F00400093E19153171F0000BD
:1000400023223FFC6FF09FFF93000000130100008C
:10005000930100001302000093020000130300004C
:100060009303000013040000930400001305000034
:10007000930500001306000093060000130700001C
:100080009307000013080000930800001309000004
:1000900093090000130A0000930A0000130B0000EC
:1000A000930B0000130C0000930C0000130D0000D4
:1000B000930D0000130E0000930E0000130F0000BC
:1000C000930F0000732540F16310050097020000B4
:1000D000938202017390523073500018970200000F
:1000E00093824202739052309B021000939252030B
:1000F0009382F2FF7390023B9302F0017390023AF5
:100100007350403097020000938242017390523046
:10011000735020307350303093010000970200007C
:10012000938282EE73905230130510001315F5017F
:10013000635C05000F00F00F930110009308D005D9
:10014000130500007300000093020000638A0200A0
:1001500073905210B7B200009B82921073902230BD
:100160007350003097020000938242017390123462
:10017000732540F1730020309300400113016000AB
:1001800033C720029303300093012000631E770CD5
:100190009300C0FE1301600033C720029303D0FF19
:1001A000930130006312770C930040011301A0FF0C
:1001B00033C720029303D0FF930140006316770AF0
:1001C0009300C0FE1301A0FF33C720029303300049
:1001D00093015000631A77089B00F0FF9390F0039F
:1001E0001301100033C720029B03F0FF9393F30326
:1001F00093016000631A77069B00F0FF9390F00371
:100200001301F0FF33C720029B03F0FF9393F30326
:1002100093017000631A77049B00F0FF9390F00342
:100220001301000033C720029303F0FF9301800005
:10023000631C7702930010001301000033C72002F3
:100240009303F0FF93019000631077029300000086
:100250001301000033C720029303F0FF9301A000B5
:1002600063147700631030020F00F00F6380010009
:100270009391110093E111009308D00513850100BB
:10028000730000000F00F00F930110009308D005D9
:100290001305000073000000731000C00000000090
:1002A000000000000000000000000000000000004E
:0C02B00000000000000000000000000042
:1010000000000000000000000000000000000000E0
:1010100000000000000000000000000000000000D0
:1010200000000000000000000000000000000000C0
:1010300000000000000000000000000000000000B0
:081040000000000000000000A8
:040000058000000077
:00000001FF
